:020000040000FA
:020000003128A5
:080008000B1D09000B11200083
:1000100048089500C60A4602031C0900C6010130C3
:10002000C706471C23282500063096002000350807
:1000300025009100250002309D0020003608250093
:1000400098002000090025000630960025000030A9
:100050009100250002309D0025000030980020000E
:10006000090021007A30990023008C0123008D01C2
:10007000210004308C00210000308D0020008C0114
:1000800020008D01210006309500200048089500D1
:100090000B110030C6008B1625000C309300250094
:1000A0000C309A00250004309E0022001D109D1483
:1000B0001D159D151D16200004309C0028000430DD
:1000C00097000030B123B8000130B123B5000230F1
:1000D000B123B6000330B123B7000930B123C80003
:1000E0000A30B123A9000B30B123AA000C30B12390
:1000F000AB000D30B123AC000E30B123AD000F309A
:10010000B123AE001030B123AF001130B123B000E5
:100110001230B123B1001330B123B2001430B12337
:10012000B3001530B123B40020008C018D01BD0156
:100130003A100830B123B900662AA201A301A40134
:10014000A501A601A701A001A1010C19B8280C194D
:10015000BA28003020020319A528203020020318F5
:10016000BE28A10A0C3021020319C128A001A5282C
:100170000000000000000000A00AA528A001A101C5
:10018000A528A001A1010C19D1280C19D3280030F1
:1001900020020319C328203020020318D728A00109
:1001A000C3280000000000000000A00AC328960138
:1001B0009701A001A101A1150C19EF280C19F12834
:1001C000003020020319DC28203020020318F52813
:1001D000A20D2214A10BED28F928A001DC280000B3
:1001E000000000000000A00ADC28A20D2210A10BD4
:1001F000ED28A001A1010C1909290C190B290030C7
:1002000020020319FB282030200203180F29A00127
:100210009D280000000000000000A00AFB28A001AB
:10022000A101A1150C1925290C192729003020023C
:10023000031912292030200203182B29A30D23149F
:10024000A10B23292F29A001122900000000000082
:100250000000A00A1229A30D2310A10B2329A0013D
:10026000A1010C193F290C19412900302002031962
:1002700031292030200203184529A0019D280000C3
:10028000000000000000A00A3129A001A101A11571
:100290000C195B290C195D2900302002031948292B
:1002A0002030200203186129A40D2414A10B592920
:1002B0006529A00148290000000000000000A00AF4
:1002C0004829A40D2410A10B5929A001A1010C1942
:1002D00075290C197729003020020319672920306D
:1002E000200203187B29A001072A0000000000005B
:1002F0000000A00A6729A001A101A1150C199129EC
:100300000C1993290030200203197E292030200285
:1003100003189729A50D2514A10B8F299B29A0014E
:100320007E290000000000000000A00A7E29A50D23
:100330002510A10B8F29A001A1010C19AB290C19C3
:10034000AD290030200203199D2920302002031816
:10035000B129A001072A0000000000000000A00A47
:100360009D29A001A101A1150C19C7290C19C929A2
:10037000003020020319B429203020020318CD29AF
:10038000A60D2614A10BC529D129A001B42900006E
:10039000000000000000A00AB429A60D2610A10B41
:1003A000C529A001A1010C19E1290C19E32900308C
:1003B00020020319D329203020020318E729A001C5
:1003C000072A0000000000000000A00AD329A001B5
:1003D000A101A1150C19FD290C19FF2900302002DB
:1003E0000319EA29203020020318032AA70D271435
:1003F000A10BFB29072AA001EA2900000000000048
:100400000000A00AEA29A70D2710A10BFB2922084A
:1004100023062406250626062706031D9D282308F5
:10042000FE39A80022082906031D202A28082A06CA
:10043000031D202A23181E2A3A10662A3A14662A17
:1004400022082B06031D2E2A28082C06031D2E2AFF
:1004500023182C2A3910662A3914662A22082D06F8
:10046000031D3C2A28082E06031D3C2A23183A2A7D
:10047000B910662AB914662A22082F06031D4A2AD3
:1004800028083006031D4A2A2318482A3911662AEB
:100490003915662A22083106031D582A2808320613
:1004A000031D582A2318562AB911662AB915662A37
:1004B00022083306031DF02A28083406031DF02AFB
:1004C0002318642A3912662A3916662A3A1C6A2ABF
:1004D0003224EC2A153038060319862A1F303806D4
:1004E00003198C2A293038060319962A2A3038062F
:1004F0000319A42A2B3038060319B22A33303806E0
:100500000319C42A343038060319D62A39188A2A1E
:100510003224EC2A9E24EC2A3918902A3224EC2A20
:10052000B918942A5C24EC2A9E24EC2A39189A2AB9
:100530003224EC2AB9189E2A4724EC2A3919A22A17
:100540005C24EC2A9E24EC2A3918A82A3224EC2AAE
:10055000B918AC2A5C24EC2A3919B02A7124EC2A87
:100560009E24EC2A3918B62A3224EC2AB918BA2A61
:100570005C24EC2A3919BE2A7124EC2AB919C22A42
:100580008724EC2A9E24EC2A3918C82A3224EC2A23
:10059000B918CC2A4724EC2A3919D02A5C24EC2A31
:1005A000B919D42A7124EC2A9E24EC2A3918DA2AA3
:1005B0003224EC2AB918DE2A4724EC2A3919E22A17
:1005C0005C24EC2AB919E62A7124EC2A391AEA2AA1
:1005D0008724EC2A9E24EC2A0030B123B8009D2801
:1005E0002209031DF52ABD019D28220803199A2B13
:1005F000A21B002B7039703A03190F2BBD019D28E7
:10060000BD019D28EC302302031D9D2807302406E0
:100610000319BC2B2508BF002408A12394283D1CE6
:10062000FE2AA5080319572B2208783A0319212B13
:100630002208743A03193F2B22087C3A0319472BEE
:100640009D28241A9D282308B123BE003223BE050D
:10065000A41D2E2B3E08031D1B249D283E080319B4
:100660001B249D2803308A0024080739820701349F
:1006700002340434083410342034403480342308E5
:10068000B1232402031D9D28BD011B249D28073092
:100690002306031D502B08302406031D182CC02BE5
:1006A0002408BF002308A123BD011B249D28221D6F
:1006B000682BA2189D28221C852B5E2B2308BB00CB
:1006C000BB030310BB0D0310BB0DBD141B249D28E1
:1006D000BD1C9D28220803393B07BC0007303C069F
:1006E0000319B72BA21D7C2B2308BF003C08A123B4
:1006F000BC01BD011B249D283C08B1232302031D1E
:100700009D28BC01BD011B249D28BD1C9D28A21D48
:10071000912B2308BF001C30A123BB01BD011B246A
:100720009D281C30B1232302031D9D28BB01BD0160
:100730001B249D2822082306031D9D283D148D019E
:100740009D282300910020003F08230093001515E9
:1007500055309600AA30960095149518AD2B2000C0
:100760000800230091001514130820000800083029
:100770002306031D182CC02B08302506031D9D28B9
:100780001F30BF000030A123FF30BF000130A12384
:10079000FF30BF000230A123FF30BF000330A12390
:1007A0000030BF000430A1230030BF000530A1237A
:1007B0005C30BF000630A1239C30BF000730A1236E
:1007C0000030BF000830A1233830BF000930A1231A
:1007D0008130BF000A30A123F830BF000B30A123C5
:1007E0008130BF000C30A123FA30BF000D30A123AF
:1007F0008130BF000E30A123FC30BF000F30A12399
:100800008130BF001030A123FE30BF001130A12382
:100810008230BF001230A123F830BF001330A12373
:100820008230BF001430A123FA30BF001530A1235D
:10083000BB013D1094288D152A242A242A242A2419
:100840002A242A248D11080000000230C300C30BA3
:10085000272C08004730C40024242E2CC40B2C2C39
:10086000000008008B1322008D172500073096002A
:100870002000370825009100250000309D0025004C
:10088000003098002800950120009A0108008B1381
:1008900022008D132500093096002000360825001F
:1008A0009100250000309D002500003098002800B0
:1008B000950120009A0108008B1322008D1325005A
:1008C0000B309600200036082500910025000030EE
:1008D0009D002500003098002800950120009A0115
:1008E00008008B1322008D1325000630960020008F
:1008F000350825009100250002309D0020003608B3
:10090000250098002800950120009A0108008B1707
:1009100022008D13250006309600200035082500A2
:100920009100250002309D00200036082500980027
:100930002800950120009A01471408008B1322001B
:100940008D13250006309600200035082500910003
:10095000250000309D0025000030980028009501FA
:1009600020009A0108001430C2003230C000C830A4
:10097000C10000000000C10BB92CC00BB72CC20B8A
:04098000B52C08008A
:020000040001F9
:02000E00A40943
:02001000FF1CD3
:10E000001F00FF00FF00FF00000000005E009C00FA
:10E01000000038008100F8008100FA008100FC0057
:0CE020008100FE008200F8008200FA007F
:00000001FF
